:100000000C9436050C947D050C946B060C947D05C0
:100010000C947D050C947D050C947D050C947D0558
:100020000C947D050C947D050C946A0D0C943C0E8B
:100030000C94EC1C0C947D050C947D050C947D05B2
:100040000C947D050C947D050C947D050C947D0528
:100050000C947D050C94601D0C947D050C947D051D
:100060000C947D050C947D050C947D050C947D0508
:100070000C947D050C947D050C947D050C947D05F8
:100080000C947D050C947D050C947D050C947D05E8
:100090000C947D050C947D050C947D050C947D05D8
:1000A0000C947D050C947D050C947D05A90ECB0E5A
:1000B000B90FCB0EB90F100F330FB90F880F9B0F6D
:1000C000B512B512E412E412421380139A159A1570
:1000D00099139A159A149A146E159A159A158515EE
:1000E00080291E1F20212223242526272D2E2A2B5E
:1000F000141A0815171C180C12132F302878041620
:1001000007090A0B0D0E0F33343579311D1B061903
:100110000511103637387D557A2C393A3B3C3D3E37
:100120003F4041424353475F6061565C5D5E5759B3
:100130005A5B62634648324445677B7F65808080B6
:100140005250514F68696A6B6C6D6E6F7071725866
:1001500000494C754A4D734B4E767C777E746654DD
:1001600046756C6C002530325820004B6579626F03
:100170006172642073746172742E0A004B65796237
:100180006F61726420696E69742E0A005B445D00C1
:100190005B435D002C035800540020006B00650099
:1001A000790062006F00610072006400200063004B
:1001B0006F006E00760065007200740065007200CA
:1001C00000000E0374002E006D002E006B002E0048
:1001D00000000403090409028D00050100A0320992
:1001E0000400000103010100092111010001224066
:1001F000000705810308000A090401000103010248
:1002000000092111010001224D00070582030800A9
:100210000A09040200010300000009211101000184
:100220002236000705830308000A090403000203BD
:1002300000000009211101000122220007058403AA
:100240002000010705040320000109040400010344
:100250000000000921110100012239000705850372
:100260002000011201100100000008EDFE126501DE
:10027000000102000105010906A101050719E02995
:10028000E715002501950875018102050819012966
:1002900005950575019102950175039101050719F1
:1002A0000029F71500250195F875018102C0063176
:1002B000FF0974A1010975150026FF009520750836
:1002C00081020976150026FF00952075089102C06D
:1002D00005010980A101850216810026B7001A8157
:1002E000002AB700751095018100C0050C0901A115
:1002F000018503160100269C021A01002A9C027542
:100300001095018100C005010902A1010901A100A8
:1003100005091901290515002501950575018102B9
:100320009501750381010501093009311581257F8A
:1003300095027508810609381581257F9501750894
:100340008106050C0A38021581257F950175088103
:1003500006C0C005010906A101050719E029E71536
:100360000025019508750181029501750881010537
:1003700008190129059505750191029501750391EB
:10038000010507190029FF150026FF0095067508CD
:100390008100C0636F6E73756D65723A20253034CD
:1003A000580A0073797374656D3A20253034580A01
:1003B000000A002530325820006B6579626F617247
:1003C000643A20004C45443A20253032580A002532
:1003D0003032583A202530386225730A00722F6374
:1003E0002030313233343536370A0064656C5F6B48
:1003F00065795F6269743A2063616E277420646571
:100400006C3A20253032580A006164645F6B65796C
:100410005F6269743A2063616E2774206164643A94
:1004200020253032580A00290A002575002F0025A2
:1004300075005D280025640020002564002000254B
:10044000640020002564007C0025303258006D6F68
:100450007573656B6579205B62746E7C782079209A
:100460007620685D287265702F61636C293A205B85
:10047000006D6B5F776865656C5F74696D655F744F
:100480006F5F6D6178203D2025640A006D6B5F779A
:100490006865656C5F6D61785F7370656564203D4C
:1004A0002025640A006D6B5F74696D655F746F5F12
:1004B0006D6178203D2025640A006D6B5F6D617869
:1004C0005F7370656564203D2025640A006D6B5F75
:1004D000696E74657276616C203D2025640A006D3A
:1004E0006B5F64656C6179203D2025640A006D6B4B
:1004F0005F776865656C5F74696D655F746F5F6D6C
:100500006178203D2025640A006D6B5F7768656522
:100510006C5F6D61785F7370656564203D20256454
:100520000A006D6B5F74696D655F746F5F6D6178F4
:10053000203D2025640A006D6B5F6D61785F7370EC
:10054000656564203D2025640A006D6B5F696E74EB
:10055000657276616C203D2025640A006D6B5F64D6
:10056000656C6179203D2025640A000A002575002C
:10057000363A20776865656C5F74696D655F746F86
:100580005F6D61783A20000A00257500353A2077C2
:100590006865656C5F6D61785F73706565643A204E
:1005A000000A00257500343A2074696D655F746F28
:1005B0005F6D61783A20000A00257500333A206D9E
:1005C00061785F73706565643A20000A00257500E4
:1005D000323A20696E74657276616C286D73293ABF
:1005E00020000A00257500313A2064656C61792885
:1005F0002A31306D73293A20000A092D2056616C8A
:10060000756573202D0A004D3E004D25643E200087
:100610003F007365742064656661756C740A0043FD
:100620003E200077686572652064656C74613A20CD
:10063000637572736F723D25642C20776865656CF5
:100640003D25640A53656520687474703A2F2F65E0
:100650006E2E77696B6970656469612E6F72672FA2
:1006600077696B692F4D6F7573655F6B6579730A79
:10067000000A092D204D6F7573656B6579202D0A71
:100680004553432F713A09717569740A313A096407
:10069000656C6179282A31306D73290A323A09690B
:1006A0006E74657276616C286D73290A333A096D30
:1006B00061785F73706565640A343A0974696D65C1
:1006C0005F746F5F6D61780A353A09776865656CAC
:1006D0005F6D61785F73706565640A363A097768A3
:1006E00065656C5F74696D655F746F5F6D61780AD5
:1006F0000A703A097072696E742076616C75657360
:100700000A643A097365742064656661756C747374
:100710000A75703A092B310A646F776E3A092D31E8
:100720000A706775703A092B31300A7067646F7709
:100730006E3A092D31300A0A7370656564203D20D8
:1007400064656C7461202A206D61785F73706565E3
:1007500064202A2028726570656174202F207469D6
:100760006D655F746F5F6D6178290A003F004D3ED3
:100770002000433E20004C25640A000A092D204336
:100780006F6E736F6C65202D0A4553432F713A09C4
:10079000717569740A6D3A096D6F7573656B65796A
:1007A0000A000A092D204D61676963202D0A643A09
:1007B0000964656275670A783A096465627567203D
:1007C0006D61747269780A6B3A09646562756720B5
:1007D0006B6579626F6172640A6D3A09646562756E
:1007E00067206D6F7573650A763A0976657273696D
:1007F0006F6E0A733A097374617475730A633A0908
:10080000636F6E736F6C65206D6F64650A302D3495
:100810003A096C61796572302D34284631302D46A5
:1008200034290A506175733A09626F6F746C6F6195
:100830006465720A6E3A094E4B524F0A003F004EF1
:100840004B524F3A206F66660A004E4B524F3A2089
:100850006F6E0A0074696D65725F72656164333230
:1008600028293A202530346C580A006B6579626F6C
:100870006172645F6E6B726F3A2025580A006B6577
:1008800079626F6172645F69646C653A2025580A09
:10089000006B6579626F6172645F70726F746F6311
:1008A0006F6C3A2025580A00686F73745F6B657926
:1008B000626F6172645F6C65647328293A20255801
:1008C0000A000A092D20537461747573202D0A00E3
:1008D0004743433A20342E392E32204156522D4C74
:1008E0004942433A20312E382E3073766E204156DD
:1008F000525F415243483A20617672350A004F50A8
:1009000054494F4E533A204C554641204D4F555374
:10091000454B45592045585452414B455920434F6A
:100920004E534F4C4520434F4D4D414E44204E4B6E
:10093000524F204B45594D41505F53454354494F09
:100940004E20343039360A004255494C443A20662C
:100950006232343834362D64697274792028323228
:100960003A32383A3432204F637420203620323005
:100970003138290A005649443A20307846454544E2
:1009800028742E6D2E6B2E29205049443A20307841
:1009900036353132285854206B6579626F61726444
:1009A00020636F6E76657274657229205645523ADF
:1009B000203078303030310A00444553433A2063C8
:1009C0006F6E76657274205854206B6579626F6122
:1009D000726420746F205553420A000A092D205674
:1009E000657273696F6E202D0A000A6D6F757365ED
:1009F0003A206F66660A000A6D6F7573653A206F5C
:100A00006E0A000A6B6579626F6172643A206F66E4
:100A1000660A000A6B6579626F6172643A206F6ED4
:100A20000A000A6D61747269783A206F66660A007E
:100A30000A6D61747269783A206F6E0A000A646503
:100A40006275673A206F6E0A000A64656275673ADC
:100A5000206F66660A000A0A626F6F746C6F6164C9
:100A600065722E2E2E2000433E20000011241FBE52
:100A7000CFEFDAE0DEBFCDBF04B603FE27C0809122
:100A8000EC039091ED03A091EE03B091EF0387305A
:100A9000904BA740B04BD1F41092EC031092ED03B1
:100AA0001092EE031092EF0314BE84B7877F84BFC9
:100AB0000FB6F894A89580916000886180936000DB
:100AC000109260000FBEE0E0F8E3099511E0A0E0AD
:100AD000B1E0E2ECFBE402C005900D92AA38B10748
:100AE000D9F723E0AAE8B1E001C01D92AC3EB207FD
:100AF000E1F70E941D0A0C94DF250C940000FF937F
:100B0000EF93E0918A01F0918B01309709F00995FC
:100B1000EF91FF910895FC018591803011F0EFDF96
:100B2000FBCF0895FF27E0E230E247FF0CC041957C
:100B300097FF09C0EDE26095709580959095611DD5
:100B4000711D811D911D27FF02C0219530E350E2E8
:100B5000AA27660F771F881F991FAA1FA41710F0D6
:100B6000A41B63955A95A9F7AA3008F0A95FA05D68
:100B7000AF93F395611571058105910541F7ED324C
:100B800011F4EF93F395F21718F43F93F395FBCF1D
:100B90008F91B5DFFA95E1F70895E991F991859183
:100BA000803021F0853219F0AADFF9CF089520E0D6
:100BB000E89455915532C1F3503311F4689455912E
:100BC0005A3348F4505390F3220F022E220F220F73
:100BD000200D250FF4CF0EF421958991999153366C
:100BE00019F3533729F1533559F1BC018827992757
:100BF000E8945C3621F48991999168945591543622
:100C000039F446EF7EF077FF0DC08FEF9FEF0AC0FB
:100C100055374AE039F0583540E121F0523642E08C
:100C200009F00895FF93EF937DDFEF91FF91B7CF28
:100C3000FF93EF93FC0181918030B9F360DFFBCF2C
:100C4000FF93EF9368DFF1CFDF93CF93CDB7DEB79C
:100C50002596A3DFCF91DF910895E9E6F0E080814A
:100C600088608083E9982F98279A2FEF89E698E18A
:100C7000215080409040E1F700C00000279858982C
:100C8000509A5998519A2FEF89EF90E02150804067
:100C90009040E1F700C000005198599A5098589A36
:100CA000E19AE99A089590910301809102018917D0
:100CB00081F0E0910001F0910101E90FF11D8081C7
:100CC0009F5F209104019223909303015098589ABA
:100CD000089580E008951F920F920FB60F9211248D
:100CE0002F933F934F935F936F937F938F939F9334
:100CF000AF93BF93EF93FF9329B1217090918D0132
:100D0000992319F0993058F403C0211108C04AC042
:100D100080918C0186952111806880938C0181E0FF
:100D2000890F80938D019830E9F560918C01809155
:100D3000020190E0AC014F5F5F4F30910401232F1F
:100D400030E0242335234091030150E02417350778
:100D500081F02091000130910101F901E80FF91FA4
:100D60006083809102018F5F9091040189238093B9
:100D700002018091020190E001962091040130E08F
:100D8000822393232091030130E08217930731F4EB
:100D90005898509A80E691E00E948B0510928D0140
:100DA00010928C01FF91EF91BF91AF919F918F9124
:100DB0007F916F915F914F913F912F910F900FBE57
:100DC0000F901F901895CF93DF93D82FD770C82F0F
:100DD000C695C695C6956D2F8C2F0E943E11811128
:100DE0000DC0EC2FF0E0E156FE4F81E090E001C035
:100DF000880FDA95EAF79081892B8083DF91CF9174
:100E00000895CF93DF93D82FD770C82FC695C69576
:100E1000C6956D2F8C2F0E943E11882371F0EC2F08
:100E2000F0E0E156FE4F81E090E001C0880FDA95D6
:100E3000EAF78095908189238083DF91CF9108958F
:100E40008091CE0381608093CE030E942D06EFE94E
:100E5000F1E080E18E0F11928E13FDCF0895CF93B4
:100E6000DF931F92CDB7DEB70E945306882309F4A3
:100E700073C09091CE0390FF0EC01F928F9325E612
:100E800031E03F932F9389830E9424060F900F90A7
:100E90000F900F90898190919E01923009F442C089
:100EA00028F4992351F09130B1F052C0933009F4F5
:100EB00043C0943009F446C04BC0803E21F0813ECF
:100EC00031F482E036C081E080939E0146C087FF06
:100ED00036C08F773AC08633D9F118F48A3229F4B4
:100EE00037C08A3AA9F1863B99F187FD0DC08C5134
:100EF000883430F4E82FF0E0E25EFE4F808101C0DC
:100F000080E00E94E30624C0E82FEF77EC51E8343C
:100F100028F4F0E0E25EFE4F808101C080E00E9494
:100F2000010716C08D3121F08D3991F484E001C0A4
:100F300083E080939E010EC0853451F485E50E94C4
:100F4000E30608C0853421F485E50E94010702C04C
:100F500010929E0181E001C080E00F90DF91CF915F
:100F60000895E82FF0E0E156FE4F80810895EFE903
:100F7000F1E080E18E0F11928E13FDCF0895089558
:100F80008091D2020895CF93DF9300D01F92CDB706
:100F9000DEB79C018091E303843019F593E09983D7
:100FA0003B832A839093E9008FEF9091E800815072
:100FB00095FD06C095ED9A95F1F700008111F5CFEA
:100FC0008091E80085FF0DC040E050E063E070E0F4
:100FD000CE0101960E945A0B8091E8008E77809393
:100FE000E8000F900F900F90DF91CF910895CF936D
:100FF000DF9300D01F92CDB7DEB72091E3032430FA
:1010000021F522E029839B838A8383E08093E90092
:101010008FEF9091E800815095FD06C095ED9A956F
:10102000F1F700008111F5CF8091E80085FF0DC038
:1010300040E050E063E070E0CE0101960E945A0B60
:101040008091E8008E778093E8000F900F900F90CA
:10105000DF91CF9108952091E3032430F1F422E051
:101060002093E9002FEF3091E800215035FD06C0B4
:1010700035ED3A95F1F700002111F5CF2091E80008
:1010800025FF0BC040E050E065E070E00E945A0B85
:101090008091E8008E778093E8000895CF93DF93E6
:1010A0002091E303243009F04AC0EC01809114013F
:1010B0008823E1F0809115018823C1F085E08093B9
:1010C000E90081E8815049F09091E80095FD05C064
:1010D0009AE29A95F1F700C0F5CF8091E80085FF7C
:1010E0002EC040E050E060E270E019C081E08093E3
:1010F000E90081E8815059F09091E80095FD07C022
:10110000EFE3F1E03197F1F700C00000F3CF8091F9
:10111000E80085FF14C040E050E068E070E0CE01D8
:101120000E945A0B8091E8008E778093E80080E25D
:10113000FE01A2EBB2E001900D928A95E1F7DF91FA
:10114000CF9108950FB607FE45C09091E303943008
:1011500009F040C09091E9009F703091EC00232F7E
:10116000217030FD20E8922B24E02093E9002091AB
:10117000EB0020FF2CC02091EE0027FF28C020911B
:10118000080130910701321709F449C03091E80095
:1011900035FF1DC0E0910501F0910601E20FF11D40
:1011A00040812F5F30910901232320930801409350
:1011B000F1002091E80025FDE2CF2091E80020FF1A
:1011C000DECF2091E8002E772093E800D8CF9F70E3
:1011D0009093E9002091070130E0B9016F5F7F4FE4
:1011E00090910901492F50E046235723609108014F
:1011F00070E04617570789F04091050150910601AC
:10120000FA01E20FF31F8083809107018F5F9091B5
:1012100009018923809307010BC08FEF0895209166
:10122000E80025FFD4CF8093F1009F709093E900F0
:1012300080E0089580E991E00E948B058091E203AF
:10124000811109C00E94EF0C0E944C0D8091E200B8
:1012500084608093E20008958CE891E00E948B0501
:101260001092E20308950895089542E061EC81E050
:101270000E94690C42E061EC82E00E94690C42E04D
:1012800061EC83E00E94690C42E261EC84E00E9420
:10129000690C42E261EC85E00C94690C8091E503F5
:1012A000833009F455C030F4813071F0823009F494
:1012B0008EC008958A3009F47AC08B3009F460C07A
:1012C000893009F09CC020C08091E403813A09F084
:1012D00096C08091E800877F8093E8008091E803C2
:1012E0009091E903892B21F460E282EB92E003C044
:1012F00060E080E090E070E00E94A50B8091E80043
:101300008B778093E80008958091E403813209F09F
:1013100076C08091E8039091E903009719F0049753
:1013200009F06DC08091E800877F8093E80080918C
:10133000E80082FD05C08091E3038111F8CF5FC012
:101340008091F1008093D2028091E8008B7753C0A6
:101350008091E403813A09F052C08091E8039091B2
:10136000E903892B09F04BC08091E800877F8093C7
:10137000E8008091E80080FFFCCF8091140136C026
:101380008091E4038132D9F58091E8039091E903DB
:10139000892BA9F58091E800877F8093E8000E945F
:1013A0009E0C8091E603809314010C94BC158091EF
:1013B000E403813221F58091E800877F8093E80083
:1013C0000E949E0C8091E7038093D3020895809140
:1013D000E403813AA1F48091E800877F8093E800DC
:1013E0008091E80080FFFCCF8091D3028093F100D0
:1013F0008091E8008E778093E8000C949E0C08950D
:10140000089508958091D2028093B1011092D20282
:1014100080E00E94BF070E94B7070C94BC150C9493
:10142000020A0E94AB1C8091E103882329F00E94EC
:10143000D41C81110C94440B0895CF9384B7877FFB
:1014400084BF0FB6F894A89580916000886180935E
:101450006000109260000FBE90E080E80FB6F89434
:1014600080936100909361000FBE82EA98E00E9431
:101470007C1C8AE091E00E94D10F8CE791E00E94F1
:101480008B050E94000A0E9492100E94EF0C0E949D
:101490004C0D8091E20084608093E200789480910A
:1014A000E3038430E1F70E9494108091CE0380FD25
:1014B00008C00E94010A8BE691E00E948B05C4E0FF
:1014C00018C081ED97E00197A1F3EFE9FFE03197B4
:1014D000F1F700C00000F7CF0E9498108091E4005F
:1014E0009091E5002091AF013091B00128173907A4
:1014F00039F48091E303853079F70E94110AF9CF1E
:101500008091E4009091E5009093B0018093AF0149
:101510008091E303843069F78091E9008F70209116
:10152000EC00922F917020FD90E8892BC093E90088
:101530009091EB0090FF43C09091EE0097FF3FC069
:101540009091080120910701291709F12091E800E5
:1015500025FF1DC0E0910501F0910601E90FF11D85
:1015600030819F5F2091090192239093080130936D
:10157000F1009091E80095FDE3CF9091E80090FF95
:10158000DFCF9091E8009E779093E800D9CF9091BB
:10159000F3002091F20030E0392B232B81F0909161
:1015A000E80090FF0CC09091E80095FF03C01092F6
:1015B000F100F9CF9091E8009E779093E8008F704A
:1015C0008093E90096CF0E94E81C8091B10180933E
:1015D000D20208950C94E30A292F332723303105D2
:1015E000C9F064F42130310581F02230310509F071
:1015F00043C08DE890E026ED31E042C02132310554
:10160000F1F02232310541F137C082E190E023E66A
:1016100032E036C099278130910541F08230910542
:1016200041F0892B49F5E2EDF1E005C0E2ECF1E093
:1016300002C0E4E9F1E0849190E09F0121C06530AF
:10164000D8F4E62FF0E0EE0FFF1FEB58FE4F20819D
:10165000318189E090E014C0653070F470E0FB01E6
:10166000EE0FFF1FE559FE4F20813181FB01EA5942
:10167000FE4F808190E004C080E090E020E030E008
:10168000FA0131832083089580E189BD82E189BD1B
:1016900009B400FEFDCF8091D8008F7D8093D800E3
:1016A0008091E00082608093E0008091E00081FD05
:1016B000FCCF0895CF92DF92EF92FF920F931F938A
:1016C000CF93DF93EC018B016A010E94BD0C811165
:1016D00033C0C114D10439F0F60180819181081B17
:1016E000190BC80FD91FE12CF12C0115110519F1A7
:1016F0008091E80085FD16C08091E8008E77809388
:10170000E800C114D10449F0F60180819181E80E0E
:10171000F91EF182E08285E00FC00E94BD0C882393
:1017200021F30AC089918093F10001501109FFEF64
:10173000EF1AFF0ADACF80E0DF91CF911F910F916E
:10174000FF90EF90DF90CF9008952091EA033091C1
:10175000EB032617370748F06115710539F420911E
:10176000E8002E772093E80001C0B90140E0611540
:101770007105A9F12091E303222309F443C0253028
:1017800009F442C02091E80023FD40C02091E80008
:1017900022FD32C02091E80020FFE9CF4091F30004
:1017A0002091F20030E0342BFC01CF01611571056E
:1017B00059F02830310540F481918093F100615057
:1017C00071092F5F3F4FF1CF41E02830310509F01B
:1017D00040E02091E8002E772093E800C8CF411127
:1017E000C9CF0AC08091E303882361F0853061F09E
:1017F0008091E80083FD0AC08091E80082FFF2CF6B
:1018000080E0089582E0089583E0089581E00895DE
:101810002091EA033091EB032617370748F0611552
:10182000710539F42091E8002E772093E80001C07B
:10183000B901FC0120E06115710591F18091E3038C
:10184000882309F440C0853009F43FC08091E80046
:1018500083FD3DC08091E80082FD2FC08091E800AB
:1018600080FFE9CF2091F3008091F20090E0922B6D
:101870006115710559F08830910540F42491209349
:10188000F1003196615071090196F2CF21E008977D
:1018900009F020E08091E8008E778093E800CBCFBC
:1018A0002111CCCF0AC08091E303882361F08530F9
:1018B00061F08091E80083FD0AC08091E80082FF1A
:1018C000F2CF80E0089582E0089583E0089581E0FA
:1018D0000895982F973058F59093E900981739F0AC
:1018E0007091EC002091ED005091F00003C0242F86
:1018F000762F50E021FF19C03091EB003E7F3093EE
:10190000EB003091ED003D7F3093ED003091EB0026
:1019100031603093EB007093EC002093ED00509316
:10192000F0002091EE0027FF07C09F5FD3CF8F709C
:101930008093E90081E0089580E008958091E403B8
:1019400087FF11C08091E80082FD05C08091E3030C
:101950008111F8CF11C08091E8008B770BC0809186
:10196000E303882349F08091E80080FFF8CF80915D
:10197000E8008E778093E80008952091E40030918C
:10198000E50095E64091EC00842F817040FF22C075
:101990008091E80080FD1CC08091E303882391F0D2
:1019A000853091F08091EB0085FD10C04091E400FE
:1019B0005091E5004217530729F39A01915011F70E
:1019C00084E0089582E0089583E0089581E0089519
:1019D00080E008954091E80042FFDECF08950E9424
:1019E0005D0D0E94650DE0EEF0E0808181608083F6
:1019F000E8EDF0E080818F77808319BCA7EDB0E03F
:101A00008C918E7F8C9380818F7E80831092E203F5
:101A100008950F931F93CF93DF930E945D0D0E9453
:101A2000650DC8EDD0E088818F77888388818068D4
:101A3000888388818F7D888319BC1092E30310927C
:101A4000DF031092E1031092E00300EE10E0F801D2
:101A500080818B7F808388818160888342E060E021
:101A600080E00E94690CE1EEF0E080818E7F80834F
:101A7000E2EEF0E0808181608083808188608083F5
:101A8000F80180818E7F8083888180618883DF91E7
:101A9000CF911F910F910895E8EDF0E080818F7E46
:101AA0008083E7EDF0E080818160808384E082BF05
:101AB00081E08093E2030C94090DE8EDF0E0808171
:101AC0008E7F80831092E20008951092DA001092C7
:101AD000E10008951F920F920FB60F9211242F93D9
:101AE0003F934F935F936F937F938F939F93AF93A6
:101AF000BF93EF93FF938091E10082FF0BC0809131
:101B0000E20082FF07C08091E1008B7F8093E100BB
:101B10000E9434098091DA0080FF1FC08091D800B4
:101B200080FF1BC08091DA008E7F8093DA00809165
:101B3000D90080FF0DC080E189BD82E189BD09B473
:101B400000FEFDCF81E08093E3030E941A0905C0E7
:101B500019BC1092E3030E942C098091E10080FFE0
:101B600019C08091E20080FF15C08091E2008E7F55
:101B70008093E2008091E20080618093E200809196
:101B8000D80080628093D80019BC85E08093E3037D
:101B90000E940F0A8091E10084FF30C08091E20032
:101BA00084FF2CC080E189BD82E189BD09B400FEBB
:101BB000FDCF8091D8008F7D8093D8008091E10087
:101BC0008F7E8093E1008091E2008F7E8093E2001F
:101BD0008091E20081608093E2008091DF0388239E
:101BE00011F084E007C08091E30087FD02C081E02E
:101BF00001C083E08093E3030E94EA0A8091E10040
:101C000083FF29C08091E20083FF25C08091E1001D
:101C1000877F8093E10082E08093E3031092DF03EB
:101C20008091E1008E7F8093E1008091E2008E7FC1
:101C30008093E2008091E20080618093E20042E0C4
:101C400060E080E00E94690C8091F00088608093E1
:101C5000F0000E943309FF91EF91BF91AF919F91E6
:101C60008F917F916F915F914F913F912F910F9045
:101C70000FBE0F901F9018951F920F920FB60F92E4
:101C800011242F933F934F935F936F937F938F9381
:101C90009F93AF93BF93CF93DF93EF93FF93C09145
:101CA000E900CF708091EC00D82FD17080FDD0E892
:101CB0001092E9008091F000877F8093F000789483
:101CC0000E94800E1092E9008091F000886080935D
:101CD000F000CD2BCF70C093E900FF91EF91DF9121
:101CE000CF91BF91AF919F918F917F916F915F91B4
:101CF0004F913F912F910F900FBE0F901F9018950D
:101D00001F93CF93DF93CDB7DEB7AA970FB6F894A2
:101D1000DEBF0FBECDBFE4EEF3E088E08E0F909102
:101D2000F10091938E13FBCF0E944E098091E80041
:101D300083FF1FC18091E4039091E503492F50E098
:101D40004A30510508F015C1FA01EA5AFF4F0C94C8
:101D5000C525803881F0823809F00BC18091E803F5
:101D60008F708093E9008091EB0085FB882780F9D4
:101D70001092E90006C08091E0039091E103911177
:101D800082609091E800977F9093E8008093F10043
:101D90001092F100C8C0282F2D7F09F0EAC08823D7
:101DA00019F0823061F0E5C08091E603813009F0DE
:101DB000E0C0933009F080E08093E1032BC0809174
:101DC000E603811127C08091E8038F7009F4D1C028
:101DD0008093E9002091EB0020FF1CC0933021F498
:101DE0008091EB00806214C09091EB009061909321
:101DF000EB0021E030E0A90102C0440F551F8A9595
:101E0000E2F74093EA001092EA008091EB008860CC
:101E10008093EB001092E9008091E800877F86C0F4
:101E20008111A7C01091E6031F778091E3008078AD
:101E3000812B8093E3008091E800877F8093E80006
:101E40000E949E0C8091E80080FFFCCF8091E3000F
:101E500080688093E300111102C082E001C083E03A
:101E60008093E30386C08058823008F082C080915E
:101E7000E6039091E7038C3D53E0950779F583E005
:101E80008A838AE289834FB7F894DE01139620E0B3
:101E90003EE051E2E32FF0E050935700E49120FF41
:101EA00003C0E295EF703F5FEF708E2F90E0EA3055
:101EB00010F0C79601C0C0968D939D932F5F24317B
:101EC00049F74FBF8091E800877F8093E8006AE27E
:101ED00070E0CE0101960E94A50B14C0AE014F5FC9
:101EE0005F4F6091E8030E94EC0ABC01892B09F462
:101EF00040C09091E800977F9093E80089819A8193
:101F00000E94080C8091E8008B778093E80031C034
:101F1000803879F58091E800877F8093E800809190
:101F2000DF038093F1008091E8008E778093E800D2
:101F30000E949E0C1EC081111CC09091E60392303D
:101F4000C0F48091E800877F8093E8009093DF03DE
:101F50000E949E0C8091DF03811106C08091E300F6
:101F600087FD02C081E001C084E08093E3030E940A
:101F700035098091E80083FF0AC08091E800877FDF
:101F80008093E8008091EB0080628093EB00AA963A
:101F90000FB6F894DEBF0FBECDBFDF91CF911F917A
:101FA00008959093D9028093D8020895E091D802C1
:101FB000F091D902309721F00190F081E02D099441
:101FC00080E00895EF92FF920F931F93CF93DF93DA
:101FD000E091D802F091D9023097B1F18C010280E2
:101FE000F381E02D09958091CE0382FF2DC080FF03
:101FF00004C089EB93E00E948B05E80110E283EBBB
:10200000E82E83E0F82E8091CE0380FF0BC08881FC
:102010001F928F93FF92EF920E9424060F900F90D1
:102020000F900F90115021961111EDCF8091CE039A
:1020300080FF0AC081EB93E0DF91CF911F910F9158
:10204000FF90EF900C948B05DF91CF911F910F9132
:10205000FF90EF900895E091D802F091D902309767
:1020600021F00480F581E02D09940895CF93DF934A
:10207000EC018091D6029091D702C817D90709F1D7
:10208000D093D702C093D602E091D802F091D90242
:102090003097B9F00680F781E02DCE010995809147
:1020A000CE0382FF0EC080FF0CC0DF93CF9383EA84
:1020B00093E09F938F930E9424060F900F900F90B0
:1020C0000F90DF91CF910895CF93DF93EC01809132
:1020D000D4029091D502C817D90709F1D093D5023F
:1020E000C093D402E091D802F091D9023097B9F0B0
:1020F0000084F185E02DCE0109958091CE0382FF09
:102100000EC080FF0CC0DF93CF9383E993E09F93D1
:102110008F930E9424060F900F900F900F90DF91E5
:10212000CF9108950C943D110E94151D0C94200729
:10213000BF92CF92DF92EF92FF920F931F93CF93B4
:10214000DF9300D000D01F92CDB7DEB70E942F07DB
:102150000BED12E0F12C8F2D0E94B107B82EF80183
:10216000C080C82639F4F3940F5F1F4FF0E1FF12CF
:10217000F2CF30C08091CE0381FD0E945911D12C45
:10218000EE24E3948E2D8C21F9F0D982FA8281E03D
:102190009E2D9B2109F480E08B830E941E1D81608F
:1021A000782F9D838C8349815A816B818D810E9418
:1021B0008F1149815A816B817C818D810E94981C8D
:1021C000F80190819E259083D394EE0CF8E0DF1205
:1021D000D9CFC9CF8FEF89838A831B820E941E1DAE
:1021E0008160782F9D838C8349815A816B818D8199
:1021F0000E948F110E94971C0E94DF1F1091DA022B
:102200000E94D60F181741F10E94D60F8093DA0270
:102210009091CE0392FF0EC090FF0CC01F928F933F
:1022200084EC93E09F938F930E9424060F900F906D
:102230000F900F908091DA020F900F900F900F90F7
:102240000F90DF91CF911F910F91FF90EF90DF9052
:10225000CF90BF900C94A91C0F900F900F900F90EF
:102260000F90DF91CF911F910F91FF90EF90DF9032
:10227000CF90BF9008950C94BF070895CF93DF933C
:102280001F92CDB7DEB769830E94B10790E021E0CD
:1022900030E0698102C0220F331F6A95E2F72823DC
:1022A000392381E0232B09F480E00F90DF91CF9157
:1022B0000895EF92FF920F931F93CF93DF938DEDCD
:1022C00093E00E948B05C0E0D0E08FE7E82E81E02C
:1022D000F82E0FEC13E08C2F0E94B1070E94811C96
:1022E000FF92EF921F928F93DF93CF931F930F93E1
:1022F0000E94240621968DB79EB708960FB6F894D3
:102300009EBF0FBE8DBFC031D10529F7DF91CF91A0
:102310001F910F91FF90EF90089508950895CF9326
:10232000DF93CDB7DEB72B970FB6F894DEBF0FBEA5
:10233000CDBF942F4F83252F588769877A878B8746
:102340004A855B85452B21F02F3F09F59F3FF9F426
:10235000DE01119686E0FD0111928A95E9F785E08C
:10236000FE01379601900D928A95E1F749815A81D5
:102370006B817C818D819E810E9499182B960FB66E
:10238000F894DEBF0FBECDBFDF91CF9108954F818E
:10239000588569857A858B850E94981CD9CFCF9303
:1023A000882309F465C0C82F8CEF8C0F813A20F088
:1023B00080E58C0F8E3248F48C2F0E9429238111E6
:1023C00057C08C2F0E94711B0CC080E28C0F88308C
:1023D00058F4C77081E001C0880FCA95EAF70E94DF
:1023E0001C1CCF910C94561C8BE58C0F833078F419
:1023F000C53A29F0C63A31F083E890E005C081E89B
:1024000090E002C082E890E0CF910C94361088E50D
:102410008C0F853168F5C83A89F0C93A91F0CA3A0B
:1024200099F0CB3AA1F0CC3AA9F0CD3AB1F0CE3A3E
:10243000B9F0CF3AC1F080E090E017C082EE90E0B2
:1024400014C089EE90E011C08AEE90E00EC085EBDA
:1024500090E00BC086EB90E008C083EB90E005C0F5
:1024600084EB90E002C087EB90E0CF910C94641075
:10247000CF910895882349F19CEF980F913A20F06D
:1024800090E5980F9E3218F40E94C41B0DC090E294
:10249000980F983058F4877091E001C0990F8A9591
:1024A000EAF7892F0E94221C0C94561C9BE5980F7A
:1024B000933020F480E090E00C943610885A8531F7
:1024C00020F480E090E00C9464100895882321F0BB
:1024D0000E941C1C0C94561C0895882321F00E9415
:1024E000221C0C94561C0895BF92CF92DF92EF925B
:1024F000FF920F931F93CF93DF9300D000D000D0B3
:10250000CDB7DEB725E0FC01DE01119601900D92FA
:102510002A95E1F7FC014081518102816381748138
:10252000258122952F706115710509F403C35F3F62
:1025300019F44F3F09F4FEC26C01862F7D836C8332
:10254000602F782F8D812E830E94F51A182FB92EB7
:102550000E94F41A0E94E419EB2DE295EF70F0E06E
:10256000E05AFF4F2E810C94C5258B2D807F9B2D2B
:102570009F70F92E882319F0F29490EFF92200232E
:1025800049F0FF2009F483C28F2D0E942F1C0E9466
:10259000561C7DC2812F0E943A12FF2009F4CAC244
:1025A0008F2D0E94351C26960FB6F894DEBF0FBE05
:1025B000CDBFDF91CF911F910F91FF90EF90DF90F2
:1025C000CF90BF900C94561C8B2D807F9B2D9F70BD
:1025D000F92E803219F0F29480EFF822112319F0CD
:1025E000113009F12AC00023B1F08F2D222351F1BF
:1025F000213041F526960FB6F894DEBF0FBECDBF51
:10260000DF91CF911F910F91FF90EF90DF90CF90CE
:10261000BF900C943F1C222319F0213009F48AC288
:102620000E94421C2DC00023F1F0263008F082C227
:102630000E94191C8F2129F023C00023F9F02111D9
:1026400016C08F2D26960FB6F894DEBF0FBECDBFF5
:10265000DF91CF911F910F91FF90EF90DF90CF907E
:10266000BF900C946612253008F064C209C0F601D0
:10267000858180FF0CC28F708583E3CF21111CC23E
:102680008F2D83C12B2D26952695237030E02115A3
:10269000310521F021303105D1F04CC2002321F069
:1026A000812F9B2D937002C080E090E026960FB69C
:1026B000F894DEBF0FBECDBFDF91CF911F910F9178
:1026C000FF90EF90DF90CF90BF900C9436100023D6
:1026D00021F0812F9B2D937002C080E090E0269620
:1026E0000FB6F894DEBF0FBECDBFDF91CF911F9123
:1026F0000F91FF90EF90DF90CF90BF900C946410FB
:10270000812F002319F00E94651E02C00E94CD1E79
:1027100026960FB6F894DEBF0FBECDBFDF91CF91E6
:102720001F910F91FF90EF90DF90CF90BF900C948E
:10273000521F8B2D837009F07BC00111FBC1812FCB
:10274000829586958770880F880F912F9F70C92E6C
:10275000D12CE12CF12C082E04C0CC0CDD1CEE1C7D
:10276000FF1C0A94D2F714FF12C04FE050E060E063
:1027700070E004C0440F551F661F771F8A95D2F77B
:10278000CB01BA01609570958095909503C060E08B
:1027900070E0CB012B2D269526952370422F50E01B
:1027A00042305105D9F04330510569F16C297D293A
:1027B0008E299F294130510551F126960FB6F89484
:1027C000DEBF0FBECDBFDF91CF911F910F91FF9064
:1027D000EF90DF90CF90BF900C94091A6C297D295F
:1027E0008E299F2926960FB6F894DEBF0FBECDBF67
:1027F000DF91CF911F910F91FF90EF90DF90CF90DD
:10280000BF900C94231A0E94091AC701B60126969C
:102810000FB6F894DEBF0FBECDBFDF91CF911F91F1
:102820000F91FF90EF90DF90CF90BF900C94EF1935
:10283000002319F08B2D817001C08695882309F43F
:1028400079C1812F829586958770880F880F912F87
:102850009F70C92ED12CE12CF12C082E04C0CC0C79
:10286000DD1CEE1CFF1C0A94D2F714FF12C04FE0CF
:1028700050E060E070E004C0440F551F661F771FF2
:102880008A95D2F7CB01BA016095709580959095A5
:1028900003C060E070E0CB012B2D269526952370B8
:1028A000422F50E042305105D9F04330510569F1D3
:1028B0006C297D298E299F294130510551F1269699
:1028C0000FB6F894DEBF0FBECDBFDF91CF911F9141
:1028D0000F91FF90EF90DF90CF90BF900C94D01AA3
:1028E0006C297D298E299F2926960FB6F894DEBF84
:1028F0000FBECDBFDF91CF911F910F91FF90EF9051
:10290000DF90CF90BF900C94E21A0E94D01AC701BA
:10291000B60126960FB6F894DEBF0FBECDBFDF918D
:10292000CF911F910F91FF90EF90DF90CF90BF90CC
:102930000C94BE1A103FD1F128F480E4810F80324C
:1029400050F0A0C0123F09F462C008F44BC0133F1E
:1029500009F472C097C0F12FF071FF2E8B2D8F718B
:10296000002351F00E94571A812FFF2019F0829501
:10297000807F68CE8F7066CE0E94781A812FFF20EC
:1029800019F08295807F01C08F7026960FB6F8945B
:10299000DEBF0FBECDBFDF91CF911F910F91FF9092
:1029A000EF90DF90CF90BF900C946D120023B1F0A8
:1029B000253008F0BFC08B2D8F7126960FB6F89486
:1029C000DEBF0FBECDBFDF91CF911F910F91FF9062
:1029D000EF90DF90CF90BF900C949D1A263008F0B6
:1029E000A9C0E9CF0023A9F08B2D8F7126960FB6D1
:1029F000F894DEBF0FBECDBFDF91CF911F910F9135
:102A0000FF90EF90DF90CF90BF900C94571A002367
:102A100059F38B2D8F7126960FB6F894DEBF0FBE3B
:102A2000CDBFDF91CF911F910F91FF90EF90DF907D
:102A3000CF90BF900C94781A002399F08B2D8F7152
:102A400026960FB6F894DEBF0FBECDBFDF91CF91B3
:102A50001F910F91FF90EF90DF90CF90BF900C945B
:102A6000421A26960FB6F894DEBF0FBECDBFDF9197
:102A7000CF911F910F91FF90EF90DF90CF90BF907B
:102A80000C943D1A0023A9F0222309F4ADCF812F25
:102A900026960FB6F894DEBF0FBECDBFDF91CF9163
:102AA0001F910F91FF90EF90DF90CF90BF900C940B
:102AB000CF11222309F4ADCF812F26960FB6F894BB
:102AC000DEBF0FBECDBFDF91CF911F910F91FF9061
:102AD000EF90DF90CF90BF900C943A124B2D4F7037
:102AE000612FC6010E94DF1D26960FB6F894DEBF47
:102AF0000FBECDBFDF91CF911F910F91FF90EF904F
:102B0000DF90CF90BF900C943D194B2D4F70612FEB
:102B1000C60126960FB6F894DEBF0FBECDBFDF917B
:102B2000CF911F910F91FF90EF90DF90CF90BF90CA
:102B30000C94E21D26960FB6F894DEBF0FBECDBFF3
:102B4000DF91CF911F910F91FF90EF90DF90CF9089
:102B5000BF9008950E943C1C0E940B1C0E94561CB2
:102B60000E9484200E94521F80E090E00E94361054
:102B700080E090E00C9464100E942C1C0C94AA1528
:102B8000CF93DF9300D000D01F92CDB7DEB7942F44
:102B90004983252F5A836B837C838D834C815D8190
:102BA000452B39F12F3F11F49F3F19F149815A818B
:102BB0006B817C818D810E94F51A292F22952F70BF
:102BC00030E02C30310504F52A3031055CF4225018
:102BD00031092230310568F4853A80F4843090F46C
:102BE000823080F0883E38F4803E60F48450813A30
:102BF00048F080E014C0803FE1F704C090E2980FF5
:102C0000983080F781E00BC02C30310521F493FB24
:102C1000882780F904C02F303105C9F3EACF0F901F
:102C20000F900F900F900F90DF91CF910895CF9359
:102C3000DF9300D000D01F92CDB7DEB70F900F907A
:102C40000F900F900F90DF91CF910895CF93DF9366
:102C500000D000D000D0CDB7DEB726960FB6F894DE
:102C6000DEBF0FBECDBFDF91CF9108951F93CF93ED
:102C7000DF93C091EB0216E08091EC02C81799F047
:102C8000D0E01C9FF0011D9FF00D1124E351FD4F7A
:102C90004081518162817381848195810E942616D1
:102CA0002196C770E9CFDF91CF911F910895409190
:102CB0001D0350911E0360911F03709120038091AA
:102CC0002103909122030C94261680912203829571
:102CD0008F7009F054C080911F03882309F44FC0FE
:102CE0008091EB02A091EC0260911D0370911E0394
:102CF0004091200350912103B6E08A1709F43FC0A8
:102D000090E041155105C1F17F3F11F46F3FA1F1F2
:102D1000B89FF001B99FF00D1124E351FD4F2181BF
:102D200072132AC02081621327C02281211124C07E
:102D3000238134812417350710F421503109241BD5
:102D4000350B283C3105C0F4209122032F702061FF
:102D50002093220326E0289FF001299FF00D1124E3
:102D6000EE50FD4F80818F70806180838DE193E014
:102D70000E9474120C94361601968770BECF089587
:102D8000BF92CF92DF92EF92FF920F931F93CF9358
:102D9000DF93CDB7DEB761970FB6F894DEBF0FBEF5
:102DA000CDBF7C0185E0F701DE011D9601900D92FB
:102DB0008A95E1F7D7014C9111965C911197129683
:102DC000DC90129713960D911C91149730911D036E
:102DD00060911E038091200390912103009709F4D4
:102DE00077C16F3F19F43F3F09F472C1B0901F03E0
:102DF000BB2009F4C5C0209122030817190728F049
:102E0000F801E81BF90BCF0104C080959095800F65
:102E1000911FCC24C394883C910580F0C12C207F65
:102E200009F0CCC0702F198B088B6D2D89890E94F9
:102E300017168DE193E00E947412B6C0822F807F36
:102E400009F047C0651314C0341312C0D11010C06C
:102E50002F702061209322030E9457168DE193E08A
:102E60000E94741280912203D70115968C932FC073
:102E70000115110519F15F3F11F44F3FF9F0CD2C09
:102E8000D1101CC08091EB022091EC0236E0821739
:102E900009F45CC090E0389FF001399FF00D1124D7
:102EA000E351FD4F6181561306C06081461303C094
:102EB0006281611103C001968770E9CFCD2CDD20BE
:102EC00009F426C180912203816080932203C12CE2
:102ED0001FC1651308C0341306C0D11004C080910F
:102EE0002203D701C9C04D875E87DF86702F198BFB
:102EF000088B6D2D89890E94C0158823E9F1DD209A
:102F0000D9F120912203822F82958F7090E0029751
:102F100074F080911D0390911E0398878F8319860A
:102F20001B870A872C87CE0107960E94741286E0C1
:102F3000F701ADE1B3E001900D928A95E1F70E94AF
:102F400065160E945716CC24C394E2C0702F198BCB
:102F5000088B60E089890E94F51A292F22952F702D
:102F600030E0223031050CF0C7C09F7009F0C1C0BD
:102F7000805E883008F4CCC0C7010E947412E3CF91
:102F80000817190708F456C0F801E81BF90BCF0120
:102F9000883C910508F453C0C12C702F198B088B05
:102FA0006D2D89890E941716EDE1F3E086E0DF01BF
:102FB0001D928A95E9F70E945716AAC0651314C09E
:102FC000341312C0D11010C080912203F701858301
:102FD000C7010E94741286E0EDE1F3E0DF011D926B
:102FE0008A95E9F7CB2C94C04D875E87DF86702FDA
:102FF000198B088B6D2D89890E94C015882309F4CF
:10300000BBCFDD2009F4B8CF20912203822F829517
:103010008F7090E002970CF48ACF80911D039091FD
:103020001E039A8389831B821D830C832E83CE010A
:1030300001967BCF80959095800F911FA9CFCD2CC5
:10304000DD2009F499CF65132EC034132CC02091D4
:10305000220320FD1FC0822F82958F70D9F0D701E7
:1030600015962C9315978F3049F08F5F982F929576
:10307000907F822F8F70892B15968C93C7010E94A9
:10308000741286E0F701ADE1B3E001900D928A95EC
:10309000E1F791CF86E0F701ADE1B3E001900D9249
:1030A0008A95E1F735C04D875E87DF86702F198BD3
:1030B000088B6D2D89890E94C015811138CF8091B0
:1030C0002203816080932203C7010E94741220C0F2
:1030D000DD2009F451CF4D875E87DF86702F198B75
:1030E000088B6D2D89890E94C015882309F444CF6F
:1030F0001ECF81113DCF0CC0243031050CF03CCFE8
:103100009F7009F435CFF7019581907F09F030CF9A
:103110008C2D61960FB6F894DEBF0FBECDBFDF9148
:10312000CF911F910F91FF90EF90DF90CF90BF90C4
:1031300008951F93CF93DF93CDB7DEB72C970FB6CB
:10314000F894DEBF0FBECDBF4F83588769877A875B
:103150008B879C87CE0107960E94C016882369F052
:103160008F8198852A853B85232BF1F19F3F09F0BC
:1031700063C08F3F09F060C037C086E0FE0137961C
:10318000DE01119601900D928A95E1F76F817885A5
:10319000EA85FB85309741F17F3F11F46F3F21F1C4
:1031A0002091EC0230E0C901019687709927409187
:1031B000EB0250E08417950709F447C069837A83CE
:1031C000FD83EC8396E0929FD001939FB00D112474
:1031D000A351BD4FFE01319601900D929A95E1F7F2
:1031E0008093EC020E94361616E08091EB029091DB
:1031F000EC028917C1F1189FC001112483519D4F22
:103200000E94C016882379F1E091EB021E9FF00125
:103210001124E351FD4F408151816281738184818A
:1032200095810E9426168091EB0290E001968770AE
:1032300099278093EB02D9CF4F81588569857A858C
:103240008B859C850E942616CFCF0E94BC151092BC
:10325000EC021092EB02EDE1F3E086E0DF011D925B
:103260008A95E9F7C1CF2C960FB6F894DEBF0FBE52
:10327000CDBFDF91CF911F910895DF92EF92FF9222
:103280000F931F93CF93DF93FC01892B09F48AC01E
:10329000E12CF12CDD24D394EF0121968491853724
:1032A00009F461C058F4843708F04EC0843008F047
:1032B0006AC08130D1F0823071F174C0883709F46E
:1032C0005DC050F4863709F455C0873709F06AC0ED
:1032D0008E2D0E94291C54C09CE7980F903708F04F
:1032E00061C08F770E943A1250C08F010E5F1F4F4E
:1032F000FE01849190E2980F983050F48770FD2D74
:1033000001C0FF0F8A95EAF78F2F0E942F1C14C06F
:103310000E94CF1113C08F010E5F1F4FFE01C49199
:1033200080E28C0F883060F4C7708D2D01C0880F4B
:10333000CA95EAF70E94351C0E94561CE80125C078
:103340008C2F0E943A12FACF9F012E5F3F4FFE0151
:10335000C491CC2369F08FE99FE00197F1F700C099
:103360000000C150F6CF9F012E5F3F4FFE01F49049
:10337000E9010BC00E94191CE82E07C00E942C1CFA
:103380000E94561C02C00E94CF118F2D882341F04D
:10339000EFE9FFE03197F1F700C000008150F6CF70
:1033A000FE017ACFDF91CF911F910F91FF90EF90A7
:1033B000DF9008956093A3037093A4038093A50303
:1033C0009093A6030C94A81C08956093A703709390
:1033D000A8038093A9039093AA030C94A71C0F93AE
:1033E0001F930091A7031091A8032091A903309186
:1033F000AA03602B712B822B932B6093A7037093EE
:10340000A8038093A9039093AA031F910F910C9492
:10341000A71C0F931F930091A7031091A80320915D
:10342000A9033091AA03602371238223932360931D
:10343000A7037093A8038093A9039093AA031F91F5
:103440000F910C94A71C0F931F930091A703109149
:10345000A8032091A9033091AA036027712782272E
:1034600093276093A7037093A8038093A903909375
:10347000AA031F910F910C94A71C60E070E0CB0190
:103480000C94DA190F931F9341E050E060E070E074
:103490008A019B0104C0000F111F221F331F8A9550
:1034A000D2F7C901B8011F910F910C94DA190F934B
:1034B0001F9341E050E060E070E004C0440F551FEE
:1034C000661F771F8A95D2F78091A3039091A4037A
:1034D000A091A503B091A6038A019B01082B192B8B
:1034E0002A2B3B2BC901B8011F910F910C94DA19BB
:1034F0000F931F9341E050E060E070E004C0440F80
:10350000551F661F771F8A95D2F740955095609595
:1035100070958091A3039091A403A091A503B0910D
:10352000A6038A019B01082319232A233B23C901EF
:10353000B8011F910F910C94DA190F931F9341E07A
:1035400050E060E070E004C0440F551F661F771F15
:103550008A95D2F78091A3039091A403A091A5032B
:10356000B091A6038A019B01082719272A273B2728
:10357000C901B8011F910F910C94DA190F931F9391
:103580000091A3031091A4032091A5033091A603F9
:10359000602B712B822B932B1F910F910C94DA19B6
:1035A0000F931F930091A3031091A4032091A503EF
:1035B0003091A60360237123822393231F910F91DF
:1035C0000C94DA190F931F930091A3031091A40395
:1035D0002091A5033091A6036027712782279327A6
:1035E0001F910F910C94DA1908958F929F92AF92C8
:1035F000BF92DF92EF92FF920F931F93CF93DF93CF
:1036000000D000D01F92CDB7DEB76B837C838D8353
:103610008A018C819D81892B21F01F3F29F44F3F26
:1036200019F480E090E04CC08B818823C9F1809030
:10363000A7039090A803A090A903B090AA0380913B
:10364000A3039091A403A091A503B091A603882A97
:10365000992AAA2ABB2A8FE1E82EF12CD501C401B0
:103660000E2C04C0B695A795979587950A94D2F726
:1036700080FF07C0DE2CB8018E2D0E94B51D01977A
:1036800029F481E0E81AF10848F7D12C88E0189F66
:10369000F0011124E00FF11DED5DFC4FD08209C057
:1036A00088E0189FF0011124E00FF11DED5DFC4F43
:1036B000D08009831A8369817A818D2D0E94B51D7E
:1036C0000F900F900F900F900F90DF91CF911F915F
:1036D0000F91FF90EF90DF90BF90AF909F908F90F1
:1036E000089590911401992321F090911501911161
:1036F00009C02091160130911701F90132969FEF10
:1037000040E030C0982F9695969596959F31A0F4FD
:10371000E0911601F0911701E90FF11D877021E08A
:1037200030E0A90102C0440F551F8A95E2F7CA0193
:103730009181892B818308959091CE0390FF23C0BE
:103740001F928F9389E094E09F938F930E942406A9
:103750000F900F900F900F9008959F3F39F04F5F9B
:103760004E3141F051915813F8CF0DC05111F7CFA0
:10377000942FF5CF9F3F39F0F901E90FF11D97FD27
:10378000FA9582830895089590911401992321F068
:1037900090911501911109C02091160130911701E6
:1037A000F9013296205E3F4F30C0982F969596953E
:1037B00096959F31A8F4E0911601F0911701E90F59
:1037C000F11D877021E030E0A90102C0440F551FB0
:1037D0008A95E2F7CA0180959181892381830895B2
:1037E0009091CE0390FF16C01F928F938BEE93E0C3
:1037F0009F938F930E9424060F900F900F900F902D
:1038000008953196E217F30729F090819813F9CFC4
:103810001082F7CF089581E090E0E0911601F091D9
:103820001701E80FF91F1082019680329105A9F760
:1038300008958091CD0308959091CD03892B8093B5
:10384000CD03089580959091CD0389238093CD0376
:1038500008958093CD0308951092CD03089590911B
:10386000CC03892B8093CC03089580959091CC0351
:1038700089238093CC0308951092CC0308958093FC
:10388000AB0308951092AB030895809116019091B7
:103890001701FC0131969C01205E3F4F80E0919121
:1038A00091118F5FE217F307D1F70895E0911601A8
:1038B000F09117018091CD038083E0911601F09182
:1038C000170190818091CC03892B80838091AB0379
:1038D000882361F0E0911601F09117019081892B06
:1038E00080830E94451C81111092AB0380911601C8
:1038F000909117010C94E20F90938B0180938A01B1
:1039000008958295982F9C7C392F36953695282FCF
:10391000237344E0249FC0011124932F982B292F57
:103920002A7A2695892F8575880F822B0895089508
:10393000CF93DF9300D000D01F92CDB7DEB70F90AA
:103940000F900F900F900F90DF91CF9108950895F1
:1039500008950C943B118091E303843021F110927F
:10396000CF0320E488E190E00FB6F894A895809307
:1039700060000FBE2093600083B7817F846083BFA7
:1039800083B7816083BF7894889583B78E7F83BF28
:103990000FB6F894A89580916000886180936000CC
:1039A000109260000FBE0895CF930E948D110E9467
:1039B0002F070E948E11C0E08C2F0E94B107811149
:1039C00004C0CF5FC031C1F701C081E0CF9108953D
:1039D0000E94B7070C94BC151F920F920FB60F925E
:1039E00011248F939F93AF93BF938091CF03811145
:1039F00013C08091D0039091D103A091D203B091D4
:103A0000D3034196A11DB11D8093D0039093D103A0
:103A1000A093D203B093D303BF91AF919F918F91A5
:103A20000F900FBE0F901F90189582E084BD93E019
:103A300095BD9AEF97BD80936E0008952FB7F894C7
:103A40008091D0039091D103A091D203B091D30380
:103A50002FBF08952FB7F8946091D0037091D103D0
:103A60008091D2039091D3032FBF0895CF92DF921C
:103A7000EF92FF920F931F932FB7F8944091D003CA
:103A80005091D1036091D2037091D3032FBF6A018B
:103A90007B01EE24FF248C0120E030E0C016D1062B
:103AA000E206F30610F4415051099A01281B390B24
:103AB000C9011F910F91FF90EF90DF90CF90089573
:103AC0001F920F920FB60F9211248F939F93AF9373
:103AD000BF938091D0039091D103A091D203B09174
:103AE000D3030196A11DB11D8093D0039093D10300
:103AF000A093D203B093D303BF91AF919F918F91C5
:103B00000F900FBE0F901F9018950E94EF0CF89425
:103B10002FEF87EA91E6215080409040E1F700C006
:103B2000000087E090EBDC018093EC039093ED03C1
:103B3000A093EE03B093EF039CE088E10FB6F894F6
:103B4000A895809360000FBE90936000FFCF28E09F
:103B5000929FF0011124E80FF11DE052FF4F949164
:103B6000892F8F7092959F700895CF93C82FCB01A6
:103B70000E94A71D282F30E080E1989FA00111240A
:103B8000422B532B4038510519F480E090E015C0CA
:103B90009770E92FF0E088E0C89FE00DF11D112437
:103BA00084E0EE0FFF1F8A95E1F7E20FF31FEE0F9F
:103BB000FF1FE050F84985919491CF91089580E0DE
:103BC00090E0089508958091D60380FF0BC0609126
:103BD0001B0185E0689FB001112475956795759567
:103BE00067952BC081FF09C060911B0185E0689F2C
:103BF000B00111247595679520C082FF07C06091C0
:103C00001B0185E0689FB001112417C09091D70374
:103C10009923D1F060911A01961788F720911B0122
:103C200085E0289F90011124929FA001939F500D41
:103C3000112470E0CA010E94B1256038710540F47A
:103C40006115710539F002C065E070E0862F0895B6
:103C50008FE7089581E008958091D60380FF08C022
:103C60006091190170E0759567957595679521C00C
:103C700081FF06C06091190170E07595679519C0C4
:103C800082FF04C06091190170E010C09091D703C9
:103C90009923C1F0609118019617A0F7809119013E
:103CA000899FC001112470E00E94B1256038710520
:103CB00028F46115710521F0862F08958FE7089586
:103CC00081E0089561E070E0F4CF803F21F40E942C
:103CD000E31D819504C0813F29F40E94E31D809378
:103CE000DA030895823F21F40E94E31D819504C008
:103CF000833F29F40E94E31D8093D9030895893FEF
:103D000019F40E942C1E05C08A3F31F40E942C1E1B
:103D100081958093DB0308958B3F21F40E942C1E34
:103D2000819504C08C3F29F40E942C1E8093DC03F3
:103D30000895843F21F48091D803816017C0853FA6
:103D400021F48091D803826011C0863F21F48091D4
:103D5000D80384600BC0873F21F48091D80388602A
:103D600005C0883F31F48091D80380618093D803E7
:103D700008958D3F21F48091D60381600BC08E3F62
:103D800021F48091D603826005C08F3F29F4809191
:103D9000D60384608093D6030895803F39F48091E0
:103DA000DA0387FF6CC01092DA0369C0813F29F4FF
:103DB0008091DA031816BCF362C09091D903823F58
:103DC00029F497FF5CC01092D90359C0833F19F4BE
:103DD0001916CCF354C0893F41F48091DB031816C7
:103DE0000CF04DC01092DB034AC08A3F29F4809149
:103DF000DB0387FF44C0F6CF8B3F39F48091DC03AF
:103E000087FF3DC01092DC033AC08C3F29F48091BB
:103E1000DC031816BCF333C0843F21F48091D8032F
:103E20008E7F17C0853F21F48091D8038D7F11C00C
:103E3000863F21F48091D8038B7F0BC0873F21F40C
:103E40008091D803877F05C0883F31F48091D803E3
:103E50008F7E8093D80313C08D3F21F48091D603C9
:103E60008E7F0BC08E3F21F48091D6038D7F05C0DD
:103E70008F3F29F48091D6038B7F8093D603809166
:103E8000D90381110EC08091DA0381110AC080919B
:103E9000DB03811106C08091DC03811102C0109206
:103EA000D70308958091CE0383FF7EC08EE494E013
:103EB0000E948B058091D8031F928F9389E494E030
:103EC0009F938F930E94240687E494E00E948B05C1
:103ED0008091D903282F082E000C330B3F938F932A
:103EE00084E494E09F938F930E94240682E494E0FC
:103EF0000E948B058091DA03282F082E000C330BCB
:103F00003F938F938FE394E09F938F930E942406B7
:103F10008DE394E00E948B058091DB03282F082E0F
:103F2000000C330B3F938F938AE394E09F938F931E
:103F30000E94240688E394E00E948B058091DC03B4
:103F4000282F082E000C330B3F938F9385E394E0CA
:103F50009F938F930E94240682E394E00E948B0536
:103F60008091D7031F928F938FE294E09F938F935A
:103F70000E9424068DE294E00E948B058091D60376
:103F80001F928F938AE294E09F938F930E9424065E
:103F900087E294E00E948B058DB79EB74C960FB6D2
:103FA000F8949EBF0FBE8DBF88ED93E00E942B104A
:103FB0000E941E1D9093D5038093D40308951F93F0
:103FC000CF93DF938091D4039091D5030E94361D47
:103FD000AC019091D703992321F020911C0130E08E
:103FE00006C020911D018AE0289F900111244217EC
:103FF000530708F485C08091D903C091DA03D091AA
:10400000DB031091DC03811107C0C11175C0D11110
:1040100073C0111171C074C09F3F19F09F5F9093DE
:10402000D703181624F40E94E31D8093D9038091CE
:10403000D90387FF05C00E94E31D81958093D903B2
:104040001C1624F40E94E31D8093DA038091DA03A6
:1040500087FF05C00E94E31D81958093DA0360917C
:10406000D903662331F1C091DA03CC2311F1062E76
:10407000000C770B880B990B0E94B82423E333E3E1
:1040800043E35FE30E941C250E9480246093D903D0
:104090006C2FCC0F770B880B990B0E94B82423E36D
:1040A00033E343E35FE30E941C250E948024609376
:1040B000DA031D1624F40E942C1E8093DB038091EA
:1040C000DB0387FF05C00E942C1E81958093DB03D4
:1040D000111624F40E942C1E8093DC038091DC03D3
:1040E00087FF05C00E942C1E81958093DC03DF9121
:1040F000CF911F910C94521F9F3F09F08FCF97CF04
:10410000DF91CF911F910895E8EDF3E085E0DF01A5
:104110001D928A95E9F71092D7031092D60308955D
:1041200081E796E00E948B051F9281E08F931F929A
:1041300085E08F9383E296E09F938F930E942406FD
:104140000F900F900F900F900F900F900895833065
:10415000E9F128F4813061F0823009F10895853069
:1041600009F462C008F449C0863009F474C00895A7
:1041700080911D01262F30E0280F311D2F3F310582
:1041800024F4680F60931D0103C08FEF80931D011D
:1041900080911D011F928F938CE595E072C08091F4
:1041A0001C01262F30E0280F311D2F3F310524F44C
:1041B000680F60931C0103C08FEF80931C018091F6
:1041C0001C011F928F938AE495E05BC080911B01D4
:1041D000262F30E0280F311D2F3F310524F4680FC2
:1041E00060931B0103C08FEF80931B0180911B0123
:1041F0001F928F9387E395E044C080911A01262F88
:1042000030E0280F311D2F3F310524F4680F6093F3
:104210001A0103C08FEF80931A0180911A011F9237
:104220008F9382E295E02DC080911901262F30E016
:10423000280F311D2F3F310524F4680F60931901B9
:1042400003C08FEF80931901809119011F928F9302
:1042500089E095E016C080911801262F30E0280FE4
:10426000311D2F3F310524F4680F6093180103C0FE
:104270008FEF80931801809118011F928F938EEE1B
:1042800094E09F938F930E9424060F900F900F90BD
:104290000F900895833081F128F4813059F08230F5
:1042A000D1F00895853009F449C0B8F1863009F499
:1042B00056C0089580911D01681720F4861B8093D5
:1042C0001D0102C010921D0180911D011F928F934C
:1042D0008FED94E054C080911C01681720F4861B78
:1042E00080931C0102C010921C0180911C011F923E
:1042F0008F938DEC94E043C080911B01681720F4EC
:10430000861B80931B0102C010921B0180911B0130
:104310001F928F938AEB94E032C080911A01681744
:1043200020F4861B80931A0102C010921A0180911A
:104330001A011F928F9385EA94E021C080911901A0
:10434000681720F4861B8093190102C0109219018E
:10435000809119011F928F938CE894E010C0809196
:104360001801681720F4861B8093180102C0109270
:104370001801809118011F928F9381E794E09F9319
:104380008F930E9424060F900F900F900F90089526
:10439000CF93C82F1F928F9386E797E09F938F93B9
:1043A0000E94240681E090E0A0E0B0E0BC01CD01D5
:1043B00004C0660F771F881F991FCA95D2F70E9405
:1043C000E5190F900F900F900F90CF910C94BC15A2
:1043D000CF938732A8F58E3108F02BC1803109F4D4
:1043E0009FC0F8F4873009F464C0A8F4863009F05F
:1043F00024C18091CE03817F8E7F8093CE038BE793
:1044000097E00E948B0587E69AE00E948B0581E089
:104410008093DE034CC08B30F1F18E3009F46CC018
:104420000CC1863109F4B0C020F4813109F4EDC02B
:1044300004C1893109F491C08B3109F449C0FDC030
:10444000883349F150F4893209F4F1C0853309F415
:10445000EEC0873209F0F1C0EAC0833409F4E7C046
:1044600028F48A3308F4E9C08953E4C0883409F099
:10447000E4C00E94BC1586E59AE00E948B052FEFF0
:1044800083ED90E3215080409040E1F700C00000B0
:104490000E94851D0CC082EA97E05CC08DE39AE023
:1044A0000E948B058091CE0381608093CE03C1E092
:1044B000C9C08091CE03C82FC17080FFEFCF89E4BF
:1044C0009AE00E948B058091CE03817F8E7F3DC054
:1044D0009091CE0391FBCC27C0F981E0C827892FAA
:1044E000C0FB81F98093CE03CC2319F080E39AE0DE
:1044F00027C082E29AE02EC09091CE0392FBCC2797
:10450000C0F981E0C827892FC0FB82F98093CE03D0
:10451000CC2319F083E19AE013C083E09AE01AC03B
:104520009091CE0393FBCC27C0F981E0C827892F57
:10453000C0FB83F98093CE03CC2351F087EF99E041
:104540000E948B058091CE0381608093CE037AC058
:104550008AEE99E00E948B05AACF8BED99E00E942C
:104560008B0589EB99E00E948B0585E799E00E9415
:104570008B0588E499E00E948B058EEF98E00E94FD
:104580008B0580ED98E0E6CF82EC98E00E948B05E9
:104590000E94D60F1F928F9388EA98E09F938F9383
:1045A0000E942406809114011F928F9381E998E064
:1045B0009F938F930E9424068091D3021F928F9322
:1045C0008EE798E09F938F930E94240680911501B7
:1045D0001F928F938BE698E09F938F930E942406FF
:1045E0000E942A1D9F938F937F936F9384E598E099
:1045F0009F938F930E9424068DB79EB746960FB661
:10460000F8949EBF0FBE8DBF52CF0E94BC15C091C3
:10461000150181E0C827C0931501CC2329F08AE455
:1046200098E00E948B050EC08FE398E093CF80E066
:1046300001C08D510E94C8213ACF8DE398E00E94BD
:104640008B05C0E08C2FCF91089580E0089580E025
:104650000895CF93C82F8091DE03813079F020F048
:10466000823009F44DC044C1E0911601F091170168
:1046700080818152823008F03DC108C0E09116016E
:10468000F091170180818152823060F48C2F0E945A
:104690002523811104C08C2F0E94E8212FC081E0C6
:1046A00090E02CC08C2F0E942723811126C0C4319A
:1046B000E1F070F4CB3081F0C031D1F40E94902051
:1046C0008EE697E00E948B0582E08093DE0315C0A2
:1046D000C93259F0C83361F48BE797E00E948B052B
:1046E00082E797E00E948B0508C01092DE0304C1A8
:1046F0008CE697E00E948B05FFC081E08170FEC0D0
:10470000C43228F5CE3108F0C1C0CB30A1F1D0F4CD
:10471000C73009F0D3C08EE180931D0182E38093FE
:104720001C018AE080931B0184E180931A0188E0D8
:104730008093190188E28093180182E196E00E943B
:104740008B05BFC0C33149F1C431C1F0B7C0CB3410
:1047500009F4A9C028F4C93289F0C83361F0AEC0A9
:10476000C13509F49EC0C23509F499C0CE3409F0B0
:10477000A5C06AE09EC00E949020A3C08091DD0386
:10478000882319F01092DD039CC08FE196E00E940F
:104790008B0581E08093DE03B1C089EF95E00E9434
:1047A0008B0587EE95E00E948B0580911D011F927D
:1047B0008F9384EE95E09F938F930E94240682EE60
:1047C00095E00E948B0580ED95E00E948B0580911D
:1047D0001C011F928F938DEC95E09F938F930E9405
:1047E00024068BEC95E00E948B058CEB95E00E94F3
:1047F0008B0580911B011F928F9389EB95E09F930E
:104800008F930E94240687EB95E00E948B0586EA31
:1048100095E00E948B0580911A011F928F9383EA85
:1048200095E09F938F930E94240681EA95E00E9471
:104830008B058CE895E00E948B05809119011F92F1
:104840008F9389E895E09F938F930E94240687E8D1
:1048500095E00E948B0580E795E00E948B05809192
:1048600018011F928F938DE695E09F938F930E947E
:1048700024068BE695E00E948B058DB79EB748967F
:104880000FB6F8949EBF0FBE8DBF1BC0CE51EC2F4C
:10489000F0E0E058FE4F80818093DD0312C061E0BC
:1048A00003C061E006C06AE08091DD030E94A7209A
:1048B00008C08091DD030E944A2103C080E196E098
:1048C00013C08091DD03882369F01F928F938AE0E3
:1048D00096E09F938F930E9424060F900F900F9065
:1048E0000F9004C087E096E00E948B0581E006C02F
:1048F0001092DE0380E002C080E000CFCF910895E7
:104900000E9487246894B1110C94162508950E9482
:10491000FB2488F09F5798F0B92F9927B751B0F032
:10492000E1F0660F771F881F991F1AF0BA95C9F733
:1049300014C0B13091F00E941525B1E008950C9497
:104940001525672F782F8827B85F39F0B93FCCF34A
:10495000869577956795B395D9F73EF490958095B0
:10496000709561957F4F8F4F9F4F0895E89409C0D0
:1049700097FB3EF490958095709561957F4F8F4F92
:104980009F4F9923A9F0F92F96E9BB279395F695A8
:10499000879577956795B795F111F8CFFAF4BB0F26
:1049A00011F460FF1BC06F5F7F4F8F4F9F4F16C08A
:1049B000882311F096E911C0772321F09EE8872F14
:1049C000762F05C0662371F096E8862F70E060E0D0
:1049D0002AF09A95660F771F881FDAF7880F969549
:1049E000879597F9089557FD9058440F551F59F032
:1049F0005F3F71F04795880F97FB991F61F09F3FCC
:104A000079F087950895121613061406551FF2CFF4
:104A10004695F1DF08C0161617061806991FF1CF44
:104A200086957105610508940895E894BB2766276B
:104A30007727CB0197F908950E942F250C94A02584
:104A40000E94922538F00E94992520F0952311F0BC
:104A50000C9489250C948F2511240C9416250E9402
:104A6000F32470F3959FC1F3950F50E0551F629F9B
:104A7000F001729FBB27F00DB11D639FAA27F00DB7
:104A8000B11DAA1F649F6627B00DA11D661F829FDE
:104A90002227B00DA11D621F739FB00DA11D621FC3
:104AA000839FA00D611D221F749F3327A00D611DE0
:104AB000231F849F600D211D822F762F6A2F1124C2
:104AC0009F5750409AF0F1F088234AF0EE0FFF1FF5
:104AD000BB1F661F771F881F91505040A9F79E3F4C
:104AE000510580F00C9489250C9416255F3FE4F362
:104AF000983ED4F3869577956795B795F795E795A2
:104B00009F5FC1F7FE2B880F911D9695879597F9AA
:104B1000089597F99F6780E870E060E008959FEF3F
:104B200080EC089500240A94161617061806090644
:104B3000089500240A941216130614060506089513
:104B4000092E0394000C11F4882352F0BB0F40F49B
:104B5000BF2B11F460FF04C06F5F7F4F8F4F9F4FDB
:104B6000089597FB072E16F4009407D077FD09D01F
:104B70000E94CB2507FC05D03EF4909581959F4F70
:104B80000895709561957F4F0895EE0FFF1F059072
:104B9000F491E02D0994AA1BBB1B51E107C0AA1F89
:104BA000BB1FA617B70710F0A61BB70B881F991FCE
:104BB0005A95A9F780959095BC01CD010895F89478
:024BC000FFCF25
:104BC2008E0100000FB2010000FFC0074E082B0843
:104BD200F707C3070101AC032808140A321E6F7AD3
:104BE20000000000000000000000000000000000C3
:104BF200000000000000007F00547C000000000064
:104C0200000000000000000055746077006100633E
:104C1200007562787172000000000000005A5B5C4F
:104C22005D5E0000005F404D36223953030603D01B
:104C320002AE027502E80101021A023302530200B7
:0A4C4200010203040506070809003B
:106800008800EA44E944E244040005000600070069
:10681000080009000A000B000C000D000E000F001C
:1068200010001100120013001400150016001700CC
:10683000180019001A001B001C001D001E001F007C
:10684000200021002200230024002500260027002C
:10685000280029002A002B002C002D002E002F00DC
:10686000300031003200330034003500360037008C
:10687000380039003A003B003C003D003E003F003C
:1068800040004100420043004400450046004700EC
:10689000480049004A004B004C004D004E004F009C
:1068A000500051005200530054005500560057004C
:1068B000580059005A005B005C005D005E005F00FC
:1068C000600061006200630064006500850067008D
:1068D000680069006A006B006C006D006E006F005C
:1068E0007000710072007300890087008A008B00BD
:1068F000E000E100E200E300E400E500E600E7007C
:00000001FF
